:100000000C941E060C94D7270C9404280C944606D6
:100010000C9446060C9446060C9446060C94460630
:100020000C9446060C9446060C94EF120C9446066B
:100030000C9446060C9446060C9446060C94460610
:100040000C9431280C9446060C941F2C0C94622CB2
:100050000C9446060C9446060C9446060C944606F0
:100060000C9446060C9446065218B4189318961829
:1000700099189C189F18A218A518B418AE18E6195C
:10008000E819E819E619E819E819E819E819E8196A
:10009000E819E819E819E819E819E819E819E81958
:1000A0006C19E819E819E819E819E819DD18E819D0
:1000B000E819E819E819E819E819E819E819E81938
:1000C000E819E819E819E819E819E8197819781908
:1000D0007819781978197819781978197819E81928
:1000E000E819E819E819E819E819DD1877197719F6
:1000F00077197719E81985198B19911997199D198D
:10010000A319A919AF19B919C319CD19D7191E19EE
:10011000E018E819E819E819E8196C19E819E8195C
:10012000E819E819E819E819E819E81976197619AB
:1001300076197619E81985198B19911997199D194E
:10014000A319A919AF19B919C319CD19D7191E19AE
:10015000E018E819E819E819E8196C191B1A1B1AB4
:100160001B1A1B1A1B1A1B1A1B1A1B1A1B1A1B1AE7
:100170001B1A1B1A1B1A311B311B311B311B311B64
:10018000311B601A6A1A741A7E1ADB1AE51AF41AFD
:10019000051B8D1CA21CAE1CB71CC61CEB1CF41C42
:1001A0003D1D061D502056205C20632071209320A9
:1001B000B120456E746572206D656E752E2E2E0011
:1001C000546F67676C6564206D6963726F50504D42
:1001D00000546F67676C656420696E76657274653C
:1001E000642050504D2100546F67676C6564205443
:1001F00058206D7574696E672100546F67676C6570
:10020000642074656C656D65747279210050726F3D
:10021000746F636F6C206572726F72207769746897
:100220002052580054696D656F7574207768656E4B
:1002300020636F6E6E656374696E6720746F205201
:100240005800507265737320616E79206B65792058
:10025000746F2063616E63656C00436F6E6E6563DF
:1002600074696E6720746F2052582C20706F776508
:100270007220757020746865205258202877697440
:10028000682062696E6420706C7567206966206EF4
:100290006F74207573696E6720616C776179732064
:1002A00062696E642900546F67676C656420276912
:1002B0006D6D656469617465206F75747075742700
:1002C00000546F67676C65642027736C61766520E6
:1002D0006D6F64652700546F67676C6564202761E4
:1002E0006C776179732062696E642700546F676769
:1002F0006C65642050504D206368616E6E656C20A3
:100300006C696D69740053657420525353492069B8
:100310006E6A656374696F6E206368616E6E656C8A
:100320002028303D3D64697361626C652900536526
:10033000742050504D206D696E696D756D20737914
:100340006E630053657420626561636F6E20696E31
:1003500074657276616C0053657420626561636FC9
:100360006E2064656C617900536574206265616319
:100370006F6E206672657175656E637920696E2097
:10038000487A3A20303D64697361626C652C205074
:10039000783D504D52206368616E6E656C20782CFC
:1003A0002046783D465253206368616E6E656C202E
:1003B00078005365742050574D2073746F7020641B
:1003C000656C61792028302064697361626C6564B2
:1003D0002C20312D323535203D3D20302E317320FB
:1003E0002D2035306D696E29005365742050504DB5
:1003F0002073746F702064656C61792028302064EC
:10040000697361626C65642C20312D323535203D75
:100410003D20302E3173202D2035306D696E29003E
:10042000536574206661696C736166652064656CF0
:1004300061792028302064697361626C65642C20C6
:10044000312D323535203D3D20302E3173202D2089
:1004500035306D696E29002A2A2A2A2A2A2A2A2A50
:100460002A2A2A2A2A2A2A2A2A2A2A2A2A2A2A2AEC
:100470002A2A2A2A0052582041636B6564202D20C5
:1004800072657665727420737563636573736675E0
:100490006C21002A2A2A2A2A2A2A2A2A2A2A2A2AAD
:1004A0002A2A2A2A2A2A2A2A2A2A2A2A2A2A2A2AAC
:1004B000002A2A2A2A2A2A2A2A2A2A2A2A2A2A2AC6
:1004C0002A2A2A2A2A2A2A2A2A2A2A2A2A2A00528E
:1004D000582041636B6564202D20757064617465DC
:1004E000207375636365737366756C21002A2A2A0D
:1004F0002A2A2A2A2A2A2A2A2A2A2A2A2A2A2A2A5C
:100500002A2A2A2A2A2A2A2A2A2A0056616C696457
:100510002063686F69636573206172653A205B319F
:100520005D2D5B31365D20286368616E6E656C20E1
:10053000312D31362900536574206F7574707574D0
:1005400020666F7220706F727420005B585D2061AE
:10055000626F7274206368616E67657320616E6498
:10056000206578697420525820636F6E6669670051
:100570005B535D20736176652073657474696E6783
:100580007320746F205258005B525D20726576654F
:1005900072742052582073657474696E6773207486
:1005A0006F2064656661756C747300557365206EA9
:1005B000756D62657273205B312D445D20746F2010
:1005C0006564697420706F727473205B452D515D92
:1005D00020666F722073657474696E677300202DD6
:1005E00020726563656976657220636F6E66696700
:1005F000757261746F722C20727820737720000AF4
:100600000A6F70656E4C52536E67200053657420FC
:1006100073657269616C2062617564726174653AB8
:10062000200056616C69642063686F696365733A82
:100630002031202D20342B34202F2032202D203823
:10064000202F2033202D20382B34202F2034202D14
:10065000203132202F2035202D2031322B34202FF5
:100660002036202D20313600536574204368616E9A
:100670006E656C20636F6E6669673A20005365741F
:100680002044617461726174652028302D32293AEA
:10069000200053657420486F70206368616E6E653A
:1006A0006C7320286D61782032342C207365706162
:1006B000726174656420627920636F6D6D61732966
:1006C0002076616C69642076616C75657320312DCC
:1006D0003235353A2000536574206368616E6E656B
:1006E0006C2073706163696E6720287831306B48C5
:1006F0007A293A200053657420524620706F77653E
:10070000722028302D37293A200053657420524634
:10071000206D6167696320286865782920652E67E8
:100720002E20307844454144463030443A2000532E
:1007300065742062617365206672657175656E63AC
:10074000792028696E20487A293A20005B5A5D207A
:10075000656E746572207265636569766572206383
:100760006F6E66696775726174696F6E2075746902
:100770006C79005B465D20646973706C61792061FF
:10078000637475616C206672657175656E63696509
:10079000732075736564005B525D2063616C6375E3
:1007A0006C6174652072616E646F6D206B65792079
:1007B000616E6420686F70206C697374005B495DC2
:1007C000207265696E697469616C697A6520736508
:1007D0007474696E677320746F20736B65746368DB
:1007E0002064656661756C7473005B585D2072658A
:1007F00076657274206368616E67657320616E64EC
:100800002065786974206D656E75005B535D20739B
:100810006176652073657474696E677320746F20E8
:10082000454550524F4D20616E64206578697420B3
:100830006D656E7500557365206E756D62657273BA
:10084000205B302D395D20746F20656469742070E1
:100850006172616D657465727300202D2053797328
:1008600074656D20636F6E66696775726174696F18
:100870006E000A0A6F70656E4C52536E672000510D
:1008800029204F7574707574206265666F726520DB
:100890006C696E6B20283D465329203A2000502970
:1008A00020536C617665206D6F64652028657870D3
:1008B0006572696D656E74616C293A20004F29205C
:1008C00054696D65642042494E44206174207374FC
:1008D000617274757020203A20004E292050504DCE
:1008E000206F7574707574206C696D69746564200F
:1008F000202020203A200044495341424C454400E6
:100900004D292050504D205253534920746F20637D
:1009100068616E6E656C202020203A20004C2920F2
:1009200050504D206D696E696D756D2073796E63E1
:10093000202875732920203A200044495341424C15
:100940004544004B29204661696C736166652062ED
:100950006561636F6E20696E74762E2028312D32AA
:10096000353573293A20004A29204661696C736144
:10097000666520626561636F6E2064656C617920D5
:1009800028302D323535203D3E20313073202D204A
:100990003135306D696E293A200049292046616958
:1009A0006C7361666520626561636F6E206672714B
:1009B0002E203A200048292050574D2073746F7024
:1009C0002064656C6179202020202020203A2000BE
:1009D00047292050504D2073746F702064656C61FE
:1009E00079202020202020203A200046292046611E
:1009F000696C736166652064656C617920202020D4
:100A00002020203A200050574D206368616E6E65AB
:100A10006C200066756E6374696F6E3A2000292041
:100A2000706F72742000506F776572546F776572C3
:100A300000445446205548462033322D62697420C4
:100A400031306368004F70656E4C52536E67525878
:100A5000206D696E6920342F36636800466C7974A6
:100A6000726F6E2F4F72616E6765525820554846FF
:100A70002038636800525820747970653A20004429
:100A8000697361626C656400487A00203D3D200016
:100A900043616C63756C61746564207061636B6540
:100AA0007420696E74657276616C3A200042292068
:100AB0004D6963726F202868616C66292050504D23
:100AC000202020203A00412920496E766572746505
:100AD000642050504D20696E20202020203A0030A4
:100AE00029204D7574652062757A7A657220286DAB
:100AF0006F73746C79293A003929205365726961E2
:100B00006C2062617564726174653A00736D617224
:100B100074506F7274004672536B79005472616E38
:100B200073706172656E740044697361626C6564B0
:100B30000038292054656C656D657472793A2020FF
:100B40002020202020003729204368616E6E656CCC
:100B500020636F6E6669673A202000362920446161
:100B60007461726174652028302D32293A2020206A
:100B700000352920486F70206368616E6E656C7364
:100B80003A2020202020003429204368616E6E65C1
:100B90006C2073706163696E673A202000332920EE
:100BA000524620706F7765722028302D37293A2001
:100BB0002020003229205246206D616769633A2067
:100BC0002020202020202020003129204261736530
:100BD000206672657175656E63793A202020000089
:100BE00000000700020100000304060000000000EE
:100BF00000000001020408102040800102040810D7
:100C00002001020408102004040404040404040263
:100C10000202020202030303030303000000002395
:100C2000002600290000000000250028002B0000FD
:100C3000000000240027002A0000502D11241FBEB0
:100C4000CFEFD8E0DEBFCDBF13E0A0E0B1E0EEEA29
:100C5000F0E602C005900D92A83CB107D9F716E066
:100C6000A8ECB3E001C01D92AE38B107E1F71CE07B
:100C7000CCE3DCE004C02297FE010E94592ECA3367
:100C8000D107C9F70E948C2D0C9455300C940000AC
:100C900080917305813019F482E08093730580910F
:100CA0007305833019F484E0809373050895A89543
:100CB0000895DC01ED91FC910190F081E02D099502
:100CC00008952091740530917505382748E0C901D1
:100CD000880F991F37FF06C09C0151E2252750E17C
:100CE000352701C09C01415091F730937505209341
:100CF0007405089588E38093760580E092ECA1E086
:100D0000B0E08093770590937805A0937905B09330
:100D10007A0587E08093830580E091EAACEBB3E34A
:100D200080937B0590937C05A0937D05B0937E0511
:100D300085E0809384058DEE9EEFADEABEED809355
:100D40007F0590938005A0938105B0938205E5E827
:100D5000F5E080E090E0863028F4DC01AE54BC4F32
:100D60002C9101C020E0219301968831910599F7DB
:100D700082E080939D058AE080939E05089580E03F
:100D80009EECADEEB4E38093BB059093BC05A093BD
:100D9000BD05B093BE0580E090E0A0E0B0E5809393
:100DA000BF059093C005A093C105B093C205E3ECC5
:100DB000F5E080E081938F5F8031E1F70895A0E056
:100DC000B0E0E5EEF6E00C94222ED82F0E948728A2
:100DD0006115710581059105C9F30E94C52E109218
:100DE0007F05109280051092810510928205C4E063
:100DF000812C912C54018A94C0907F05D09080055D
:100E0000E0908105F0908205FE2CED2CDC2CCC24AA
:100E10000E94C02EA50194010E94012E6C0D7D1D23
:100E20008E1D9F1D60937F057093800580938105C3
:100E300090938205C15001F7DD2309F450C005E805
:100E400015E0E801A12CB12C62E3C62ED12CE12CD7
:100E5000F12C8881882309F442C0B39419F40E94CC
:100E60007A063DC00E94C02EA70196010E94012E65
:100E7000E1E0E60FA5E8B5E08A2F801B8A1520F493
:100E80008D918E13F9CFE9CF2091840530E0A0E158
:100E9000B7E20E94992D9B01AC01AE2FB0E00E94F9
:100EA000A82D40907B0550907C0560907D0570904A
:100EB0007E05640D751D861D971D4090BB055090E5
:100EC000BC056090BD057090BE05461657066806C5
:100ED000790618F2E993A39488E1A812BACFCDB7A6
:100EE000DEB7E0E10C943E2E8436910520F4BC017F
:100EF00080E090E017C09C018E3B910528F42A55B4
:100F00003109AAE0B0E00CC0823D910528F4245BD1
:100F10003109A4E6B0E004C02D5C3109A8E5B2E0D7
:100F20000E94992DA4E6B0E09B01AC010E94A82D7F
:100F3000089590E08C599F4F0E947407089561E0D6
:100F40008FE00E94342960E08FE00E946D290895AF
:100F5000892B11F061E001C060E08FE00E946D29F3
:100F6000089560E08CE00E94342961E08BE00E94EB
:100F7000342961E08DE00E94342960E082E00E9423
:100F8000342961E084E00E943429089542E050E071
:100F900068E476E080E00E94B7270895E3E0F0E09F
:100FA00089E080935700E491E67081E0E63009F033
:100FB00080E00895CF93DF93C82F0E94CE07882347
:100FC00081F0DFB781E080937205F8940E945706A4
:100FD00088E180936000C0936000C1110E945706B1
:100FE000DFBFDF91CF9108958F929F92AF92BF9212
:100FF000CF92DF92EF92FF92CF93FC01C0A5EC2F2E
:10100000E770F0E0E658FC4FA081B0E0C7FF03C0F6
:1010100024E130E002C02FE030E0FC0197A183E141
:10102000989FF0011124E25CFE4F80809180A280A5
:10103000B380A20FB31F20E43FE14DE750E00E94D0
:10104000B32DA50194010E94DF2D8C2F887149F4E6
:1010500069017A01E0EDCE0EE7E0DE1EE11CF11C35
:101060001BC0C7FF05C060E47AE88CE29EE004C0C4
:1010700060E07EEE8AEB9BE069017A01F8EBCF0E2F
:10108000FBE0DF1EE11CF11CA50194010E94DF2D95
:10109000C20ED31EE41EF51EC701B60169517C4F76
:1010A0008F4F9F4F28EE33E040E050E00E94DF2D4D
:1010B000A8EEB3E00E94A82DCF91FF90EF90DF90B3
:1010C000CF90BF90AF909F908F9008958F3F9105E4
:1010D00051F048F0811522E0920738F081159340D5
:1010E00030F482E0089580E0089581E0089583E07F
:1010F0000895A0E0B0E0EFE7F8E00C942B2EEB01B0
:101100008A01B82FB695A0E028813981F8012083A3
:101110002A813B8121832C813D8122832E813F8145
:101120002383688179814A815B812C813D81EE81B5
:10113000FF819F2F9295990F990F907C272F2370F5
:10114000922B252F2370220F220F922B232F2370F7
:101150002295207F922BF80194830B5F1F4F2896D6
:10116000AF5FBA1788F680FF24C0888199810E94FA
:101170006608D82E8A819B810E946608E82E8C81A1
:101180009D810E946608F82E8E819F810E946608CC
:10119000F0E4DF9EA001112490E1E99E900111246A
:1011A000242B282BE4E0FE9EB0011124262BF8010D
:1011B0002083CDB7DEB7E7E00C94472E803223E0E2
:1011C000920708F1883E23E0920740F48F51934044
:1011D000E4E096958795EA95E1F70895803D27E04C
:1011E000920718F48C5D93400895883928E092079F
:1011F00068F4885C974074E0969587957A95E1F756
:101200008D509C4F089580E090E008958FEF93E01B
:1012100008958C30910540F4A4E0880F991FAA9599
:10122000E1F7885D9C4F0895843F23E0920718F40E
:1012300084529C4F0895811524E0920740F486570C
:10124000934FF4E0880F991FFA95E1F7089580E92C
:1012500098E008959C013695279525753575821B74
:10126000930B9C0123733373969587959695879579
:1012700083739373820F931F9C0154E036952795D7
:101280005A95E1F7280F391F2F703F7041E051E068
:10129000249FC001259F900D349F900D1124892F0C
:1012A00008952D98882319F000002B9A02C00000A1
:1012B0002B9800002D9A000008952D9A000083B10C
:1012C0002D980000829581700895CF93DF93D82FD9
:1012D0005C9A2D985C98C8E08D2F80780E94510907
:1012E000DD0FC150C9F72D98DF91CF9108958F7709
:1012F0000E9465090895CF93DF93D82FC8E08D2F02
:1013000080780E945109DD0FC150C9F72D98DF91F7
:10131000CF910895CF93DF932D98C8E080E0D82F28
:10132000DD0F0E945D098D0FC150C9F7DF91CF918C
:1013300008950E9477090E948A095C9A0895A1E0A5
:10134000B0E0E5EAF9E00C94302E806869830E94F1
:1013500065096981862F0E947B095C9A2196E2E0EB
:101360000C944C2ECF93C0917F05C827E82FF0E056
:10137000EA58FA4F678589E70E949F096C2F8DE331
:101380000E949F096C2F82E40E949F09CF910895CB
:1013900086E20E9499090895CF93DF93EC016C8156
:1013A0008CE10E949F096D818DE10E949F096E81F1
:1013B0008EE10E949F096F8180E20E949F096885EB
:1013C00081E20E949F09698582E20E949F096A85E5
:1013D00083E20E949F096B8584E20E949F096C85CD
:1013E00085E20E949F096D858AE20E949F096E85B1
:1013F0008EE60E949F096F858FE60E949F0968898B
:1014000080E70E949F09698981E70E949F096A8994
:1014100082E70E949F09DF91CF910895CF92DF92DA
:10142000EF92FF92CF93DF936B017C01C11488E3AD
:10143000D8068CE9E8068CE1F80628F5C701B60164
:1014400020E836E948E950E00E94DF2DE90168977D
:1014500060E879E687E69FEF0E94BB2D6C0D7D1D4D
:101460008E1D9F1DF2E0660F771F881F991FFA954A
:10147000D1F721E732E040E050E00E94DF2DF22E6C
:10148000E32E80E421C0C701B60120E03DE241E344
:1014900051E00E94DF2DE901689760E073ED8EEC6A
:1014A0009EEF0E94BB2D6C0D7D1D8E1D9F1D660F36
:1014B000771F881F991F21E732E040E050E00E942B
:1014C000DF2DF22EE32E80E66C2F6F71680F85E71B
:1014D0000E949F096E2D86E70E949F096F2D87E766
:1014E0000E949F09DF91CF91FF90EF90DF90CF9006
:1014F0000895682F8DE60E949F0908958F929F920C
:10150000AF92BF92CF92DF92EF92FF92CF93DF9391
:10151000D82F83E00E9499098093710584E00E948E
:1015200099098093700560E086E00E949F0961E060
:1015300087E00E949F096FE789E00E949F0965E0AC
:101540008AE00E949F0962E18BE00E949F0965E1A9
:101550008CE00E949F096DEF8DE00E949F0960E082
:101560008EE00E949F09DD2319F08BE291E008C014
:1015700020919D0533E1239FC0011124825C9E4F81
:101580000E94CC096CE880E30E949F096FE082E32F
:101590000E949F0962E483E30E949F0980919E0557
:1015A00087FF02C064E101C06AE084E30E949F09F2
:1015B0006AE285E30E949F096DE286E30E949F092B
:1015C00064ED87E30E949F0960E088E30E949F0921
:1015D00060E089E30E949F09D11109C0C0907F0596
:1015E000D0908005E0908105F090820507C0C5E9A4
:1015F000CC2EC1ECDC2EED2CCEEDFC2ECAE38F2CD4
:101600009924AA24BB24682D8C2F0E949F09682D41
:1016100085E08C0F0E949F09FE2CED2CDC2CCC2445
:10162000CF5FCE3361F76FEF83E40E949F096FEFC6
:1016300084E40E949F096FEF85E40E949F096FEF89
:1016400086E40E949F09DD2311F066E002C06091EC
:1016500083058DE60E949F0960E089E70E949F094B
:10166000609184058AE70E949F0960E083E70E94F9
:101670009F0960E084E70E949F09D11109C0609131
:101680007B0570917C0580917D0590917E0504C05D
:1016900060E071EA8CEB93E30E940E0ADF91CF9138
:1016A000FF90EF90DF90CF90BF90AF909F908F9082
:1016B000089561E087E00E949F0964E28EE70E943E
:1016C0009F0963E088E00E949F0960E088E00E9433
:1016D0009F0965E087E00E949F0962E085E00E9423
:1016E0009F0983E00E9499098093710584E00E941C
:1016F000990980937005089583E00E949909809369
:10170000710584E00E9499098093700561E087E08B
:101710000E949F096AE070E080E090E00E94AA28A1
:101720000E94590B00000895CF92DF92FF920F9311
:101730001F93CF93DF931F92CDB7DEB7082F162FDD
:101740008EE399830E949F09F02EC02E9981D92E95
:101750008C2D8F19811738F4F60161916F018FE795
:101760000E949F09F5CF64E085E00E949F0983E015
:101770000E9499098093710584E00E9499098093E1
:1017800070050E94872860936C0570936D058093A7
:101790006E0590936F0569E087E00E949F0981E0E4
:1017A000809373050F90DF91CF911F910F91FF9060
:1017B000DF90CF9008950F931F930E94940B809118
:1017C0007305813099F40E94872800916C0510916F
:1017D0006D0520916E0530916F05601B710B820BBA
:1017E000930B603A76488140910548F380917305E8
:1017F000813031F46EE971E082EE95E00E94732A47
:101800001F910F9108950F931F938091730582305C
:1018100021F41092730581E020C08091730581301E
:10182000D9F40E94872800916C0510916D052091D4
:101830006E0530916F05601B710B820B930B613A43
:1018400076488140910540F061E087E00E949F0961
:101850001092730582E001C080E01F910F910895FE
:10186000CF93DF93EC014AE050E06D2F70E082EE01
:1018700095E00E94412B6EE282EE95E00E94452A9F
:10188000BE0184E0769567958A95E1F76F707727BA
:101890004AE050E082EE95E00E94412B6EE282EE3B
:1018A00095E00E94452ABE016F7077274AE050E01C
:1018B00082EE95E00E94412BDF91CF910895D82FC1
:1018C000C0E0CD1790F45E9A409A64E670E080E044
:1018D00090E00E94AA285E98409864E670E080E05C
:1018E00090E00E94AA28CF5FECCF6CE271E080E02C
:1018F00090E00E94AA28E4CF0F931F93CF93DF9329
:10190000EC01062F15E0115051F0CE010E943C3041
:10191000081741F0602FCE010E944430F4CF82E0DE
:101920000E945F0CDF91CF911F910F910895A0E06D
:10193000B0E0EDE9FCE00C94222E482E562EC0E0DB
:10194000D0E0612C712CE12CF12C00E010E0411072
:101950000CC06090D40586E4689E3001112459E1E2
:10196000E52EF12C0AEB15E01EC091E049120FC0E4
:101970006090D405E6E46E9E30011124FBE16F0E09
:10198000711C49E2E42EF12C06E715E00CC082E060
:10199000481209C028E1622E77247394EE24E39460
:1019A000F12C03ED15E043018C0E9D1E1092750580
:1019B000109274053401A62CA818B12CC30101960D
:1019C0006C01AE14BF04A8F4A00EB11E511006C0E5
:1019D000C3010E943C30F501808305C0F5016081A0
:1019E000C3010E947C0CF50180810E9461063601D2
:1019F000E2CFC301511018C0C3010E943C30B82E81
:101A0000C6010E943C302B2D30E0322F2227282B9C
:101A100080917405909175058217930779F4C0E061
:101A2000D0E05524539493CF3601609175050E9400
:101A30007C0C60917405C6010E947C0CC05EDE4F78
:101A4000C13E92E0D90708F482CF852DCDB7DEB72D
:101A5000E0E10C943E2E61E082E00E94970C089534
:101A600060E082E00E94970C8091D305853020F0E1
:101A70001092D3050E942B0D8091D3058093D4053D
:101A8000089561E080E00E94970C61E081E00E948F
:101A9000970C089560E080E00E94970C882351F035
:101AA00060E081E00E94970C882321F08091760508
:101AB000883349F00E94BF060E947A0681E00E94A6
:101AC000DF060E94410D0895882319F06AEA71E04B
:101AD00002C06EEA71E082EE95E00E94732A0895DA
:101AE000FF920F931F93CF93DF9369EC7BE082EE1D
:101AF00095E00E941F2A40917B0550917C056091E2
:101B00007D0570917E052AE030E082EE95E00E942E
:101B1000482B63EB7BE082EE95E00E941F2A409108
:101B20007F0550918005609181057091820520E1CB
:101B300030E082EE95E00E94482B6DE97BE082EE7A
:101B400095E00E941F2A4AE050E06091830582EEF2
:101B500095E00E94702B67E87BE082EE95E00E94A2
:101B60001F2A4AE050E06091840582EE95E00E94D1
:101B7000702B61E77BE082EE95E00E941F2AC5E8AA
:101B8000D5E0F12C8E0188818823A9F0FF2031F067
:101B900061EB71E082EE95E00E94422A21964AE0D4
:101BA00050E0F801608182EE95E00E94392BF394B9
:101BB000F8E1FF12E7CF82EE95E00E944D2A6BE537
:101BC0007BE082EE95E00E941F2A4AE050E060919F
:101BD0009D0582EE95E00E94702B66E47BE082EE2C
:101BE00095E00E941F2AE0919E05E770F0E0EE0F5D
:101BF000FF1FEE57FC4F6081718182EE95E00E94DD
:101C0000732A61E37BE082EE95E00E941F2A8091B7
:101C10009E058871883069F028F4811113C068E24C
:101C20007BE00CC0803141F0883161F46CE07BE0F6
:101C300005C06CE17BE002C066E17BE082EE95E0EE
:101C40000E94612A68EF7AE082EE95E00E941F2AE6
:101C500040917705509178056091790570917A05EA
:101C60002AE030E082EE95E00E94482B6FED7AE0AA
:101C700082EE95E00E941F2A8091BF0580710E942C
:101C8000640D66EC7AE082EE95E00E941F2A809156
:101C9000BF0580740E94640D6DEA7AE082EE95E0E3
:101CA0000E941F2A8091BF0580720E94640D60E926
:101CB0007AE082EE95E00E941F2A86E795E00E9476
:101CC000F407AB01BC012AE030E082EE95E00E940F
:101CD0002A2B6BE87AE082EE95E00E941F2A86E7C5
:101CE00095E00E94F4079B01AC0160E472E48FE090
:101CF00090E00E94DF2DBA01A9012AE030E082EED7
:101D000095E00E942A2B68E87AE082EE95E00E9436
:101D1000612ACDB7DEB7E5E00C94492E8F929F92F1
:101D2000AF92BF92CF92DF92EF92FF92811107C0E4
:101D30006FE77AE082EE95E00E94612A2FC090E082
:101D40000E94740724E630E040E050E00E94DF2D5E
:101D5000CA01B9012AE030E040E050E00E94DF2DE6
:101D600049015A016B017C012AE030E0B501A40170
:101D700082EE95E00E942A2B6EE282EE95E00E94B0
:101D8000452A2AE030E0B701A60182EE95E00E94E4
:101D90002A2B63E782EE95E00E94852AFF90EF9060
:101DA000DF90CF90BF90AF909F908F9008951F933A
:101DB000CF93DF9365E77AE082EE95E00E941F2AD9
:101DC00080919F05813041F46CE57AE082EE95E0E8
:101DD0000E94612A10E050C0823019F465E47AE074
:101DE000F5CF843019F461E37AE0F0CF853091F7D4
:101DF00066E27AE0EBCFC12FD0E0C930D1050CF418
:101E000041C068E3610F82EE95E00E94452A6EE1D1
:101E10007AE082EE95E00E941F2ABE016F5F7F4F3D
:101E20004AE050E082EE95E00E94092B63E17AE0FF
:101E300082EE95E00E941F2AC156DA4FE981E03216
:101E400018F566E07AE082EE95E00E941F2A89810B
:101E5000803130F06DE673E082EE95E00E94422A18
:101E600069816F7070E06F5F7F4F4AE050E082EEF3
:101E700095E00E94122B1F5F80914805181708F407
:101E8000BACF0FC061E3BECFEF70F0E0EE0FFF1FDF
:101E9000EE56FC4F6081718182EE95E00E94732ABC
:101EA000EACF6BEE79E082EE95E00E941F2A8091E6
:101EB000B7050E948E0E60ED79E082EE95E00E94FB
:101EC0001F2A8091B8050E948E0E65EB79E082EEA4
:101ED00095E00E941F2A8091B9050E948E0E6AE942
:101EE00079E082EE95E00E941F2A4091AF05509163
:101EF000B0056091B1057091B205411551056105BC
:101F0000710539F12AE030E082EE95E00E94482B1D
:101F100067E679E082EE95E00E941F2A8091B30582
:101F20000E949907AB01BC012AE030E082EE95E007
:101F30000E94482B63E479E082EE95E00E941F2A1C
:101F40004AE050E06091B40582EE95E00E94702B6B
:101F500006C06AE379E082EE95E00E94612A6DE1B5
:101F600079E082EE95E00E941F2A6091B50570919C
:101F7000B6054AE050E082EE95E00E945A2B60E000
:101F800079E082EE95E00E941F2A6091AE056034F0
:101F900050F470E06F5F7F4F4AE050E082EE95E0D2
:101FA0000E94122B06C067EF78E082EE95E00E9457
:101FB000612A6AED78E082EE95E00E941F2A809106
:101FC000AD0580FF03C063EB71E002C067EB71E019
:101FD00082EE95E00E94732A6DEB78E082EE95E048
:101FE0000E941F2A8091AD0582700E94640D6EE9E7
:101FF00078E082EE95E00E941F2A8091AD05847002
:102000000E94640D6FE778E082EE95E00E941F2A3F
:102010008091AD0588700E94640DDF91CF911F9172
:1020200008950F931F93CF93DF93209145052F3F82
:10203000A9F56FEF75E082EE95E00E941F2A81E816
:1020400093E00E94300C6EED75E082EE95E00E9408
:102050001F2A80914605909147050E94300C6BEA3B
:1020600075E082EE95E00E94612A68E875E082EEF4
:1020700095E00E94612A60E775E082EE95E00E949B
:10208000612A6BE475E082EE95E00E94612A82EE9F
:1020900095E00E944D2A0E94D70E68C012160CF0DF
:1020A00065C0332727FD30958091480590E0821761
:1020B00093070CF45BC066E375E082EE95E00E9446
:1020C0001F2A60914505772767FD70954AE050E02B
:1020D00082EE95E00E94122B6BE075E082EE95E0B7
:1020E0000E941F2A10E008E2809149051817D0F5D8
:1020F000C12FD0E0CC0FDD1FC65BDA4F288130E066
:1021000080914505992787FD9095019728173907F4
:1021100039F56BEB71E082EE95E00E94422A4AE0CD
:1021200050E0602F82EE95E00E94392B6FEB71E05A
:1021300082EE95E00E94422AE981EF70F0E0EE0F16
:10214000FF1FEE56FC4F6081718182EE95E00E9488
:10215000422A63EC71E082EE95E00E94422A0F5F12
:102160001F5FC2CF82EE95E00E944D2ADF91CF9192
:102170001F910F910895FF920F931F93CF93DF93B9
:10218000C5E8D5E0F12C8E0188818823D1F165EC7A
:1021900071E082EE95E00E94422A4AE050E06F2D05
:1021A00082EE95E00E94392B62ED71E082EE95E0BF
:1021B0000E94422A2196F801208130E0A0E1B7E296
:1021C0000E94992D9B01AC01A0918405B0E00E9472
:1021D000A82DAB01BC0180917B0590917C05A0915D
:1021E0007D05B0917E05480F591F6A1F7B1F2AE0AD
:1021F00030E082EE95E00E94482BF394F8E1FF1264
:10220000C2CFCDB7DEB7E5E00C94492E1092DF04C3
:1022100085E6E0EEF4E0DF011D928A95E9F7089586
:10222000CF93C82F8F3719F0883009F045C0E0915F
:10223000DF04EE23D9F1E150E093DF04F0E0E05257
:10224000FB4F10826DE070E082EE95E00E9459062F
:10225000C0E08091DF04C81760F4EC2FF0E0E0529A
:10226000FB4F608170E082EE95E00E945906CF5FDF
:10227000F0CF60E270E082EE95E00E9459066DE0DA
:1022800070E082EE95E00E945906C0E08091DF0484
:10229000C81778F5EC2FF0E0E052FB4F608170E05A
:1022A00082EE95E00E945906CF5FF0CF67E082EEA4
:1022B00095E00E94452A1DC08B3119F40E94061139
:1022C0001AC08D30C1F08A30B1F08091DF048436BD
:1022D00068F76C2F70E082EE95E00E945906E0915D
:1022E000DF0481E08E0F8093DF04F0E0E052FB4FCB
:1022F000C08380E001C081E0CF910895CF93C82FC3
:102300000E9487286093C8047093C9048093CA040C
:102310009093CB04C093DD04CC2329F040E051EE30
:1023200060E070E004C040E855E260E070E082EEFA
:1023300095E00E94CF2CCF9108959091CC04492F25
:102340004F7050E0BA016F5F7F4F292F30E0E4E01B
:1023500035952795EA95E1F76217730759F0FA0169
:10236000E353FB4F808381E0890F8F70907F892B2F
:102370008093CC0408956EE770E082EE95E00E94B1
:1023800059060895A3E1B1E0E8ECF1E10C94232EA5
:10239000E5E8F5E0712C8191882321F0739428E120
:1023A0007212F9CF66ED71E082EE95E00E94732A19
:1023B0004AE050E0672D82EE95E00E94702B80E0AD
:1023C0000E947E0A0E94590B8E010E5F1F4FC12C86
:1023D000D12C7601C39466246A945C2C0E947B28DD
:1023E0004B015C012091840530E0A0E1B7E20E943E
:1023F000992D9B01AC01C701B6010E94BB2D209114
:102400007B0530917C0540917D0550917E05620FE2
:10241000731F841F951F2091BB053091BC0540910F
:10242000BD055091BE05261737074807590718F410
:10243000F801608229C08C2D0E94B20961E070E031
:1024400080E090E00E94AA28F80110820E947B2878
:10245000681979098A099B09643F714081059105D2
:1024600040F40E94C809F8019081981778F780839A
:10247000EDCF50FE05C05D9841985E9A409A04C029
:102480005D9A419A5E9840982FEFC21AD20AE20AEA
:10249000F20A0F5F1F4F8FEFC816D104E104F10459
:1024A00009F09BCFCE019395FC01D82E7FEF68EC0D
:1024B0002E2F281B271510F051E056C0DE01129672
:1024C00051E02FEF41E03D91321710F0322F01C063
:1024D000452F5F5F5F3F11F0232FF5CF4193242FEE
:1024E00030E0A1E0B0E0AC0FBD1FA20FB31F5C93C2
:1024F000413079F0DE01A20FB31F5C93423049F006
:10250000AFEFBFEFAC0FBD1FA20FB31F6C934E3FD9
:1025100078F6A2E0B0E0AC0FBD1FA20FB31F7C9312
:102520004D3F30F6A3E0B0E0AC0FBD1FA20FB31FCC
:102530006C93BECF452F242F30E0FC01E20FF31F38
:102540006081AFEFB0E0AC0FBD1FA20FB31F2C91A5
:10255000621748F44150DC01A40FB11D2C91208377
:102560006C934111E8CF5F5F571520F3372D3695F7
:1025700020E0231770F4DC01A20FB11D4C91522F03
:10258000530FFC01E50FF11D50815C9340832E5FDA
:10259000F0CFF5E8EF2EF5E0FF2E8C01802F8D199E
:1025A000871598F4F801C1908F014AE050E06C2D36
:1025B00082EE95E00E94392B6CE282EE95E00E945B
:1025C000452AF701C1927F01E9CF82EE95E00E9492
:1025D0004D2A81E0CD5EDE4FEFE00C943F2E1F923E
:1025E0000F920FB60F9211241F932F933F934F9387
:1025F0005F936F937F938F939F93AF93BF93CF938B
:10260000DF93EF93FF93C0918600D0918700809174
:102610008704909188042091A904211155C09E013E
:10262000281B390B8091BF059091C005A091C10571
:10263000B091C20585FD02C036952795253C49E03D
:102640003407B8F140910A0150E060E070E02CE1FD
:10265000B695A795979587952A95D1F70097A105E7
:10266000B10521F481E090E0A0E0B0E08417950787
:10267000A607B707D8F480910A018F3FB9F040E070
:1026800080910A01481780F4842F90E0880F991FE9
:10269000FC01E757FB4F20813181FC01E55FFE4FD4
:1026A000318320834F5FECCF1092AA0410920A016D
:1026B0000BC02D3B82E0380720F080910A01803169
:1026C000D8F08FEF80930A01D0938804C0938704D9
:1026D000FF91EF91DF91CF91BF91AF919F918F913A
:1026E0007F916F915F914F913F912F911F910F902B
:1026F0000FBE0F901F90189510910A0181E0810F75
:1027000080930A01C9010E94DE08E12FF0E0EE0F7C
:10271000FF1FE757FB4F91838083D6CF83E08093E1
:1027200080008AE9809381008091BF0586FD05C005
:10273000809181008064809381008FEF9FEF909360
:1027400089008093880080916F00806280936F0081
:1027500008950E94300D8091D405843011F41092B8
:10276000D40508956F3018F086958058089589E053
:10277000689F802D11240895A0E0B0E0E2ECF3E121
:102780000C942A2EC82F0E9487280091380410919B
:10279000390420913A0430913B046B017C01C01A4A
:1027A000D10AE20AF30A9701860149E8C41643E117
:1027B000D406E104F10410F010923C046093380454
:1027C0007093390480933A0490933B042091A904B8
:1027D0008FEF820F8230D8F5E0913C04EE2309F4AC
:1027E0004EC1E13011F482E0B8C1E03108F034C1EB
:1027F00081E08E0F80933C04F0E0E757FB4FC083ED
:10280000803109F0ACC1EBE8F4E0213029F4A1817A
:10281000A695A695808108C080819181A92FA69553
:10282000A695A69596958795A03148F4B0E090E0DE
:10283000AA0FBB1FA55FBE4F11969C938E9310925B
:10284000AA04329684E0E939F807F9F688C1233002
:1028500009F005C1E0913C04E11104C0CF3009F05A
:102860007EC10DC1E83148F481E08E0F80933C04B5
:10287000F0E0E857FB4FC08372C1E83109F0ECC0CB
:10288000C111EAC040E050E0ABE0CA01B3E0880FFC
:10289000991FBA95E1F7A49F9001A59F300D1124CF
:1028A000F901E757FB4F6081E1817E2F77707595C5
:1028B0006795FC01EE0FFF1FE55FFE4F718360839C
:1028C000F901E657FB4FB081B695B695B695E18113
:1028D000FE2FF295FF0FF07E6F2F6B2BE695E6959E
:1028E000E6957E2F777075956795FC01EE0FFF1FBB
:1028F000E35FFE4F71836083F901E557FB4FB081C1
:10290000B295B695B695B370C181DC2FDD0FDD0FA2
:102910006D2F6B2BC295C695C695C370E281E17091
:10292000EE0FEE0F7E2F7C2B75956795FC01EE0F59
:10293000FF1FE15FFE4F71836083F901E357FB4F97
:10294000B081B695E181FE2FF795FF27F7956F2FA0
:102950006B2BE6957E2F777075956795FC01EE0FD2
:10296000FF1FEF5EFE4F71836083F901E257FB4F5B
:10297000B081B295BF70E181FE2FF295F07F6F2F8D
:102980006B2BE295EF707E2F777075956795FC0144
:10299000EE0FFF1FED5EFE4F71836083F901E1577B
:1029A000FB4FB081BB1FBB27BB1FC181DC2FDD0FDD
:1029B0006D2F6B2BCC1FCC27CC1FE281E370EE0F69
:1029C0007E2F7C2B75956795FC01EE0FFF1FEB5E4C
:1029D000FE4F71836083F901EF56FB4FB081B695CE
:1029E000B695E181FE2FF295FF0FFF0FF07C6F2F60
:1029F0006B2BE695E6957E2F777075956795FC01B4
:102A0000EE0FFF1FE95EFE4F71836083F901EE5602
:102A1000FB4F20812295269527703181E32FEE0F01
:102A2000EE0FEE0F6E2F622B732F729576957770E7
:102A300075956795FC01EE0FFF1FE75EFE4F7183F2
:102A400060834F5F5F4F4230510509F01ECF809188
:102A50009F0483FF1092AA0410923C0480C024308B
:102A600009F07DC060913C0461110BC0C83AB1F41B
:102A7000109275051092740588EA0E94610681E043
:102A80006CC0613019F4C093370404C0623031F473
:102A9000C09336048C2F0E9461065AC0E091360420
:102AA0002E2F30E0220F331F462F50E0C90102962F
:102AB000841795073CF0633268F7FA01EA57FB4F39
:102AC000C083E8CF2D5F3F4F8C2F90E0609174055D
:102AD000709175054217530749F4982F8827862768
:102AE0009727909375058093740532C0681779070E
:102AF00069F580913704813049F5E13118F080E1C2
:102B000080933604F0903604CAE8D4E000E010E088
:102B10000F15D0F4FE013197808190E0982F88271F
:102B20002881822B63E0969587956A95E1F70E944C
:102B3000DE08F801EE0FFF1FE55FFE4F91838083F3
:102B40000F5F1F4F2296E4CF1092AA0410923C040C
:102B500080913C04882319F08F5F80933C04CDB7AB
:102B6000DEB7E8E00C94462EE82FF0E0E654FA4F8A
:102B7000E185E03150F4F894F0E0EE0FFF1FE55FDF
:102B8000FE4F8081918178940895E03121F0E13108
:102B900031F483E101C082E10E94C929089580E0F7
:102BA00092E00895A2E2B0E0E8EDF5E10C94202E69
:102BB0009E012F5F3F4F80E1D9011D928A95E9F771
:102BC00064E072E082EE95E029A33AA30E94732AA2
:102BD0000E947C0B1D8A1E8A1F8A188E312C212C84
:102BE00000E0812C912C5401412C74E7572E7BE896
:102BF000672E72E3772EE0E5CE2EE3ECDE2EE12C9D
:102C0000F12C84EF91E0A0E0B0E08D8F9E8FAF8F2C
:102C1000B8A380E09EECADEEB4E3898F9A8FAB8FC2
:102C2000BC8F80E094E7ABE8B2E3898B9A8BAB8BE7
:102C3000BC8B82EE95E00E94872B892B09F4E1C0C2
:102C400082EE95E00E94B42B9C0133272C32310593
:102C500009F442C0ACF42332310509F0ABC019824B
:102C60001A821B821C821D821E821F821886198670
:102C70001A861B861C861D861E861F86188A60C0C3
:102C80002434310529F02335310509F4B2C092C04E
:102C900064E482EE95E00E94452A2AE030E040E0BC
:102CA00054E76BE872E382EE95E00E94D32A6CE26F
:102CB00082EE95E00E94452A2AE030E040E05EEC9A
:102CC0006DEE74E382EE95E00E94D32A6CE282EE10
:102CD00095E00E94852AADCF0F5F043009F0A9CF9F
:102CE00029813A814B815C81A8EEB3E00E94A82D36
:102CF000698B7A8B8B8B9C8B2D813E814F81588584
:102D00000E94A82D698F7A8F8B8F9C8F29853A8599
:102D10004B855C852D8F3E8F4F8F58A32D853E852B
:102D20004F8558890E94A82D6B017C0160323EE4DA
:102D300073078105910530F462E38CE10E949F09DD
:102D400000E077CF603345E774078105910510F403
:102D500062E2F3CF60345CE975078105910510F4F8
:102D600066E2EBCF80E5C81683ECD806E104F104F7
:102D700010F462E1E2CF90E6C9169AEED906E104BA
:102D8000F10410F465E1D9CFA0E7CA16A1E1DA0693
:102D9000A1E0EA06F10410F461E0CFCFB0EACB166F
:102DA000B6E8DB06B1E0EB06F10410F463E0C5CF52
:102DB00065E0C3CF10ED180F1A3008F03ACFE1E00C
:102DC000F0E0EC0FFD1F24E0029FE00DF11D112447
:102DD0002081318142815381AAE0B0E00E94A82D78
:102DE000610F711D811D911D6083718382839383A7
:102DF00020CF49885A886B887C88812C912C54017B
:102E000018CF81149104A104B10489F4C301B20163
:102E10000E940E0A61E070E080E090E00E94AA2823
:102E20001D8A1E8A1F8A188E312C22242A948D8D89
:102E30009E8DAF8DB8A188169906AA06BB06D0F460
:102E40000E94C8092D893E894F89588D280F311D50
:102E5000411D511D2D8B3E8B4F8B588F381608F41A
:102E6000382E821508F4282E3FEF831A930AA30AFE
:102E7000B30A56C0C301B20128EE33E040E050E08F
:102E80000E94DF2DBA01A9012AE030E082EE95E030
:102E90000E942A2B6CE282EE95E00E94452A4AE0CD
:102EA00050E0632D82EE95E00E94392B6CE282EEB9
:102EB00095E00E94452A6D897E898F89988DA501AC
:102EC00094010E94DF2DBA01A9012AE030E082EED0
:102ED00095E00E942A2B6CE282EE95E00E94452A42
:102EE0004AE050E0622D82EE95E00E94392B6CE2C0
:102EF00082EE95E00E94852A4C0C5D1C6E1C7F1CA6
:102F0000898D9A8DAB8DBC8D84159505A605B70569
:102F100020F449885A886B887C88812C912C540134
:102F200029893A894B895C89283E334041055105FE
:102F300009F07FCEA296E2E10C943C2EACE1B0E029
:102F4000E4EAF7E10C942A2E0E9487286B017C01A9
:102F500081E00E947E0A14E703E0198361E0CE015C
:102F600001960E94DB0B009373050E94590B6AEFD8
:102F700070E080E090E00E94AA2880917305833081
:102F800089F482EE95E00E94872B892B59F40E94E8
:102F900087286C197D098E099F096038734C894C0C
:102FA0009140D8F280917305833009F44FC08FE7C8
:102FB0000E9477090E948A098983843511F083E091
:102FC0005CC00E948A0910924605809347050E94C2
:102FD0008A092091460530914705280F311D30930D
:102FE0004705209346050E948A09809348050E9460
:102FF0008A0980934905813110F7F12C0F2D10E0DB
:103000008091490590E0880F991F0817190740F42F
:103010000E948A09F801E65BFA4F8083F394EECFB1
:1030200080E7898361E0CE0101960E94DB0B83E09B
:10303000809373050E94590B62E370E080E090E09A
:103040000E94AA2880917305833011F482E015C094
:103050008FE70E9477090E948A098983803509F0E9
:10306000AECF0FE915E00E948A09F80181938F0124
:10307000F5E00A3B1F07B9F781E06C96E8E00C9495
:10308000462E80914505992787FD9095A92FB92F48
:10309000FC013196EB30F10508F066C0EC5CFF4FA7
:1030A0000C94572E62E778E082EE95E00E94612A48
:1030B00081E893E00E94300C6AE578E082EE95E0CA
:1030C0000E94612A65E378E082EE95E00E94612A21
:1030D0006BE078E082EE95E00E94612A6AEE77E08C
:1030E00082EE95E00E94612A6DEB77E082EE95E03A
:1030F0000E94612A67E977E082EE95E00E94612AEA
:1031000063E777E082EE95E00E94612A6CE477E065
:1031100082EE95E00E94612A82EE95E00E944D2A9F
:103120000E94700D21C06FE277E01AC06AE077E07C
:1031300017C065EF76E014C066ED76E011C062E975
:1031400076E00EC06DE776E00BC068E676E082EED2
:1031500095E00E94612A62E276E002C06CE076E0CF
:1031600082EE95E00E94612A6AE070E080E090E0E3
:103170000E94AA2882EE95E00E94872B892B29F0D5
:1031800082EE95E00E94B42BF5CF0895ACE1B0E05B
:10319000ECECF8E10C942A2E909145059F3F09F044
:1031A00023C1482F50E0FA013A97EF36F10508F0B5
:1031B0000FC1E15CFF4F0C94572E61E172E0A0C09B
:1031C0006DE172E082EE95E00E94732A85E78983C3
:1031D0008BE1EFE9F5E0DE01129601900D928A9500
:1031E000E1F76CE1CE0101960E94DB0B0E94590BC6
:1031F00083E08093730568EC70E080E090E00E94CB
:10320000AA2880917305843009F0E2C08FE70E94FC
:1032100077090E948A098983853509F0D9C06DEE46
:1032200074E082EE95E00E94612A6FEC74E082EE19
:1032300095E00E94612A61EB74E096C065E372E05C
:1032400082EE95E00E94732A89E6898361E0CE01CF
:1032500001960E94DB0B0E94590B83E0809373055B
:1032600068EC70E080E090E00E94AA2880917305ED
:10327000843009F0ADC08FE70E9477090E948A0967
:1032800089838E010E5F1F4F7E014DE1E40EF11C1C
:103290000E948A09F80181938F01EE15FF05C1F79D
:1032A0008BE1FE013296AFE9B5E001900D928A956F
:1032B000E1F78981893409F08BC063E974E082EE1B
:1032C00095E00E94612A65E774E082EE95E00E9435
:1032D000612A67E574E048C06FE472E082EE95E031
:1032E0000E94732A8EEF8093450572C080528750EA
:1032F000805390914805981708F066C06EE572E01B
:1033000082EE95E00E94732A63C084E180934505B4
:1033100060E274E029C085E18093450569EE73E0C1
:1033200023C086E18093450562EB73E01DC087E111
:103330008093450568E673E017C088E180934505F2
:1033400067E573E011C089E18093450563E473E0AC
:103350000BC08AE1809345056EE273E005C08BE106
:103360008093450566E073E082EE95E00E94612A55
:103370002FC06CEE72E082EE95E00E94612A80918F
:10338000AD0591E01DC066ED72E082EE95E00E9411
:10339000612A8091AD0592E013C061EC72E082EE8B
:1033A00095E00E94612A8091AD0594E009C066EA2B
:1033B00072E082EE95E00E94612A8091AD0598E06E
:1033C00089278093AD058FEF809345050E941110EA
:1033D00082EE95E00E94872B892B09F45AC182EE78
:1033E00095E00E94B42BF4CF0E941011882309F4B9
:1033F00050C18091DF04811104C08FEF8093450597
:1034000040C140E050E060E070E080EE94E00E9457
:10341000CE2E40914505042F112707FD1095212F31
:10342000312FF8013197EB31F10508F01AC1E2555F
:10343000FF4F0C94572E552747FD50952091480576
:1034400030E0241735070CF40CC18B019C010150AE
:10345000110921093109003211052105310558F002
:10346000C0904905EBE4F5E0F12CD12CA8E2EA2E5E
:10347000415051090FC0FA01E156FA4F6150608383
:10348000D8C0DF0111972C9130E02417350729F0BF
:10349000F3943296FC10F5CFCAC00E2D10E020E058
:1034A00030E0061717072807390741F42081DA01B1
:1034B000A156BA4F11962C93DD24D394E394E8CF10
:1034C0006F3F71058105910511F008F0CAC0609346
:1034D000B705AFC06F3F71058105910511F008F088
:1034E000C0C06093B805A5C06F3F71058105910507
:1034F00011F008F0B6C06093B9059BC02091E004BC
:1035000020622037E9F440E050E060E070E081EEB6
:1035100094E00E94CE2E9B01AC01DC01CB0101970F
:10352000A109B1090897A105B10508F0ADC0A4ED46
:10353000B0E30E94A82D6A5E7C4A8A46954E24C05C
:103540002636E9F440E050E060E070E081EE94E07F
:103550000E94CE2E9B01AC01DC01CB010197A10999
:10356000B1090797A105B10508F08EC0A8EAB1E638
:103570000E94A82D645E7C438E46944E05C0611562
:1035800071058105910571F08B019C0114572B4841
:1035900032430130FAE51F07F2E62F07F2E03F075A
:1035A00008F05FC06093AF057093B0058093B105DC
:1035B0009093B2053EC06F3F71058105910511F0F2
:1035C00008F04FC06093B30534C08B019C010150DB
:1035D0001109210931090F3F11052105310508F0B5
:1035E00040C06093B40525C08B019C01045C194068
:1035F000210931090D344DE114072105310528F465
:103600007093B6056093B50514C061157105810509
:10361000910521F48FEF8093AE050BC061347105E5
:1036200081059105F0F461506093AE0502C0DD2084
:10363000C1F08091DE0481111AC080917F059091C4
:103640008005A0918105B09182050196A11DB11D53
:1036500080937F0590938005A0938105B0938205A8
:1036600006C060E772E082EE95E00E94732A0E9435
:1036700006118FEF809345056AE082EE95E00E9487
:10368000852A0E94111005C061E070E080E090E0A2
:103690007BCF6C96E8E00C94462E6AE572E082EEF1
:1036A00095E00E94612A62E472E082EE95E00E9459
:1036B000612A82EE95E00E94872B892B31F082EE01
:1036C00095E00E94B42B0E94C6180E949E1782307B
:1036D00029F0833051F46DE072E002C064E272E0E0
:1036E00082EE95E00E94612A08958FEF8093450550
:1036F0001092DE040E941110809145058E3F69F002
:1037000082EE95E00E94872B892BB1F382EE95E043
:103710000E94B42B0E94C618EFCF08950F931F93F9
:10372000109145051F3F09F0D2C0893409F457C0F4
:1037300000F5883309F469C058F4803309F477C080
:1037400008F061C08B3109F440C08132B1F1B9C0D9
:10375000813409F487C030F4893309F466C08034B9
:1037600061F1AFC0823409F48EC0863409F448C0D8
:10377000A8C0823609F487C078F4883531F128F47E
:103780008235C1F18335E1F09CC08A3509F494C0DB
:10379000813609F467C095C0823761F128F4863616
:1037A00079F18936E1F08DC0883779F08A3709F4EC
:1037B00083C0833709F085C003C061E172E015C0A2
:1037C0000E94410D6EE872E004C00E944A0D68EA52
:1037D00072E082EE95E00E94732A8EEF70C00E9424
:1037E0007A060E94BF0667EC72E082EE95E00E94C6
:1037F000732A67C081E00E94DF0660EE72E0F5CFB9
:103800000E94BB105EC080535AC06AEF71E082EE26
:1038100095E00E94612A90919E0588E0890F887149
:10382000977E892B80939E051AC089E048C067EE79
:1038300071E082EE95E00E94612A8091BF0590912F
:10384000C005A091C105B091C20520E182278093F7
:10385000BF059093C005A093C105B093C205109316
:1038600045052FC061ED71E082EE95E00E94612A6E
:103870008091BF059091C005A091C105B091C2058E
:1038800040E4842710C060EC71E082EE95E00E9475
:10389000612A8091BF059091C005A091C105B091AA
:1038A000C20520E282278093BF059093C005A093B4
:1038B000C105B093C20502C00E944D1B8FEF8093DB
:1038C0004505809145058E3F09F0D4C0DDC00E94BA
:1038D0001011882309F4D8C08091DF04811104C03D
:1038E0008FEF80934505C6C040E050E060E070E097
:1038F00080EE94E00E94CE2E00914505112707FD31
:103900001095212F312FF8013197E930F10508F09A
:10391000B4C0E753FF4F0C94572E8B019C0101500C
:1039200014472B4832430F3F19452246324008F0D6
:10393000A4C060937B0570937C0580937D05909374
:103940007E0577C060937F05709380058093810525
:103950009093820581E08093DE046BC0683071052E
:103960008105910508F089C06093830562C08B01D1
:103970009C0101501109210931090A301105210565
:10398000310508F07AC06093840553C061EB71E0A3
:1039900080EE94E00E94083010E0009799F00E94B9
:1039A000E22F009779F0183130F4E12FF0E0EA5877
:1039B000FA4F87871F5F61EB71E080E090E00E9423
:1039C0000830EBCF1831A8F5E12FF0E0EA58FA4FB4
:1039D00017861F5FF7CF653071058105910508F0E7
:1039E0004CC060939D0525C08B019C0101501109BD
:1039F000210931090630110521053105F0F5209125
:103A00009E05287F262B20939E0513C08B019C01C9
:103A100001501109210931090115124C21403105CC
:103A200060F560937705709378058093790590939E
:103A30007A058091DE04811113C080917F059091F9
:103A40008005A0918105B09182050196A11DB11D4F
:103A500080937F0590938005A0938105B0938205A4
:103A60000E9406118FEF809345056AE082EE95E093
:103A70000E94852A0E94411807C060E772E082EE2A
:103A800095E00E94732AECCF1F910F9108958FEF5C
:103A9000809345051092DE040E94411880914505EF
:103AA0008E3F69F082EE95E00E94872B892BB1F35F
:103AB00082EE95E00E94B42B0E948E1BEFCF6AE04D
:103AC00070E080E090E00E94AA2882EE95E00E94DB
:103AD000872B892B29F082EE95E00E94B42BF5CF3D
:103AE0000895CF93C82F682F82EE95E00E94E12BB6
:103AF00090916A059C2790936A05CF910895A1E063
:103B0000B0E0E5E8FDE10C94302E99830E94711D30
:103B10009981892F0E94711D2196E2E00C944C2E10
:103B20001F93CF93DF93182FEB0110926A0565EB7B
:103B300070E082EE95E00E94590662E670E082EE47
:103B400095E00E945906812F0E94711DCE010E94AE
:103B50007F1DDF91CF911F91089560916A0582EEDC
:103B600095E00E94E12B0895A1E2B0E0EAEBFDE1CF
:103B70000C942C2E7B018A018C3009F453C108F07F
:103B800040C0863009F4BCC018F5833009F491C0F8
:103B900070F4813009F472C0823009F048C26BE1E0
:103BA00070E082E00E94901D0FE915E078C084303B
:103BB00009F487C0853009F03AC26091490570E088
:103BC000660F771F85E00E94901D0AE415E086C00D
:103BD000893009F4A7C070F4873009F49BC088309D
:103BE00009F025C261E070E088E00E94901D80919C
:103BF000D40523C28A3009F4CAC08B3009F4F2C05C
:103C000016C28A3609F475C1D8F4873609F43AC168
:103C100038F4853609F40EC1863609F41FC107C28F
:103C2000883609F437C1893609F001C261E070E0D5
:103C300089E60E94901D0E947A060E94BF06F5C187
:103C40008D3609F4D4C138F48B3609F491C18C3621
:103C500009F49AC1ECC18E3609F4DCC1873C09F045
:103C6000E6C161E070E087EC0E94901D81E00E9457
:103C7000711D0E94AD1D10926B05E3C169E270E0F9
:103C800081E00E94901D06E715E0F80181918F0107
:103C90000E94711DF5E00F391F07B9F7D0C1F80177
:103CA00081918F010E94711DF5E00A3B1F07B9F752
:103CB000C6C161E070E083E00E94901D0E949E17E3
:103CC000BCC161E070E084E00E94901D81E00E9430
:103CD000711D0E94AD1D0E94D215B3C1809149058E
:103CE00090E0880F991F98012A543540281739070A
:103CF00008F0A5C1F80181918F010E94711DEECFDE
:103D000062E070E086E00E94901D81E893E00E94EE
:103D10007F1D95C161E070E087E00E94901D809159
:103D200048058BC186E6898361E0CE0101960E9439
:103D3000DB0B0E94590B83E08093730568EC70E005
:103D400080E090E00E94AA28809173058430D9F425
:103D50008FE70E9477090E948A098983863469F473
:103D600060E270E089E00E94901D10E20E948A09E2
:103D70000E94711D1150D1F762C161E070E089E0CD
:103D80000E94901D52C161E070E089E053C169E179
:103D900070E08AE00E94901D81E08093BA05209136
:103DA00072058091BF059091C005A091C105B091A9
:103DB000C205222311F0806801C08F778093BF0570
:103DC0009093C005A093C105B093C2050AEB15E01E
:103DD000F80181918F010E94711DF5E0033D1F07DD
:103DE000B9F72DC161E270E08BE00E94901D8091D7
:103DF000AA048F3F39F08091AA0491E0980F909324
:103E0000AA0402C08091AA040E94711D10E0812FB3
:103E10000E94B4150E9409090E947F1D1F5F103186
:103E2000B1F70DC161E070E08CE00E94901D8091BF
:103E3000D30503C161E070E085E60E94901D89E230
:103E4000E816F10409F0F8C0D801E6E7F5E08D9135
:103E5000819385E0EF39F807D1F7E7C061E070E0C2
:103E600086E60E94901DEBE1EE16F10409F0E4C035
:103E7000D801EFE9F5E08D91819385E0EA3BF80701
:103E8000D1F7D3C061E070E087E60E94901D0E94E8
:103E9000410DCBC061E070E088E60E94901D85E78F
:103EA00089838BE1EFE9F5E0DE01129601900D9236
:103EB0008A95E1F76CE1CE0101960E94DB0B0E942E
:103EC000590B83E08093730560E273E080E090E03B
:103ED0000E94AA2880917305843009F0ADC08FE755
:103EE0000E9477090E948A098983853509F0A4C058
:103EF0009CC061E070E08AE60E94901D89E689839B
:103F000061E0CE0101960E94DB0B0E94590B83E019
:103F10008093730560E273E080E090E00E94AA283D
:103F200080917305843009F087C08FE70E9477097C
:103F30000E948A0989838E010E5F1F4F7E01EDE189
:103F4000EE0EF11C0E948A09F80181938F01EE1593
:103F5000FF05C1F78BE1FE013296AFE9B5E00190B4
:103F60000D928A95E1F78981893409F065C05DC0B9
:103F700061E070E08BE60E94901DF80180818093E3
:103F8000D4050E944A0D51C061E070E08CE60E94A9
:103F9000901DF0E2EF16F10461F487E6898380E278
:103FA000F801DE01129601900D928A95E1F761E227
:103FB00003C087E4898361E0CE0101960E94DB0B98
:103FC0000E94590B83E0809373056CE474E080E0F9
:103FD00090E00E94AA2880917305843069F58FE7EC
:103FE0000E9477090E948A09873431F51EC061E07A
:103FF00070E08DE60E94901D89E1E816F104E1F47D
:10400000D801EAEBF5E08D91819385E0E33DF80777
:10401000D1F70BC061E070E08EE60E94901DF801C0
:1040200080818093D3050E942B0D81E006C061E062
:1040300070E08AEC0E94901D80E00E94711D0E9439
:10404000AD1DA196E6E00C94482EA0E0B0E0EBE2B6
:10405000F0E20C942A2ECAECD3E014E606E035E038
:10406000F32E44E0E42E53E0D52E62E0C62E82EE1D
:1040700095E00E94872B892B09F49BC082EE95E086
:104080000E94B42B282F809335044091340450E0D3
:104090004730510560F7FA01EE52FF4F0C94572E4E
:1040A000853B29F781E080933404E1CF823609F023
:1040B0007DC0C0923404DBCF8093330480933204FC
:1040C000D0923404D4CF9C01332730933104209311
:1040D000300490913204982790933204E092340493
:1040E000C6CF382F22274091300450913104242B21
:1040F000352B30933104209330049091320498276B
:1041000090933204F09234042536310508F4AFCF91
:1041100061E070E08CEC0E94901D81E00E94711DB6
:104120000E94AD1D43C020912E0430912F04F9014F
:10413000E653FC4F80839091320498279093320489
:10414000C901019690932F0480932E04209130048E
:10415000309131048217930708F489CF0093340417
:1041600086CF8091320482130BC060912E0470912F
:104170002F044AEC53E0809133040E94B41D0DC01B
:1041800062E070E08BEC0E94901D809133040E94ED
:10419000711D80916A050E94711DFE01812F11928F
:1041A0008A95E9F710922F0410922E04109234048D
:1041B0005ECFCDB7DEB7E8E00C94462E81E0809369
:1041C0006B0580916B05882349F082EE95E00E9493
:1041D000872B892BB1F30E942520F3CF0895AAE203
:1041E000B0E0E5EFF0E20C94282E0E947B286B01F2
:1041F0007C0181E00E947E0A82EE95E00E94872B7E
:10420000892B29F082EE95E00E94B42BF5CF5E98C1
:10421000409811E072E6B72EE9E2AE2E03E00E946C
:104220007B286C197D098E099F09693C7105810500
:104230009105E0F11123D1F10E947B286B017C01F3
:104240005D9A419A80ED97E00E94A807B982E6E75F
:10425000F5E0DE0112968A2D01900D928A95E1F724
:104260006AE2CE0101960E94DB0B5D98419880E0E6
:1042700090E00E94A807009373050E94590B62E327
:1042800070E080E090E00E94AA288091730584305D
:1042900061F4009373058FE70E9477090E948A09F1
:1042A00011E0823419F410E001C011E083E10E94B2
:1042B000A029892BA1F411E012C05E9A409A5D9A60
:1042C000419A82EE95E00E94B42B8D309105B9F0B1
:1042D0006CF40A97A1F05E9840985D98419882EE40
:1042E00095E00E94872B892B41F799CF8332910566
:1042F00079F08234910579F70E94DE20ECCF62EBF1
:1043000071E082EE95E00E94612A0E94471DE3CF92
:104310000E94D215E0CF8F929F92AF92BF92CF9220
:10432000DF92EF92FF921F93CF93DF9383E10E947E
:10433000A029892B09F089C068EC70E080E090E04A
:104340000E94AA2880E090E00E94A8070E947B2893
:104350004B015C016B017C0180ECC80E82E1D81E30
:10436000E11CF11C0E947B286C157D058E059F05C4
:1043700030F483E10E94A029892BA1F364C083E17A
:104380000E94A029892B09F05EC080ED97E00E9471
:10439000A8070E947B286B017C01D0E0C1E088E483
:1043A000880E86E2981EA11CB11C11E083E10E94D8
:1043B000A029892B21F58C149D04AE04BF0430F490
:1043C00080ED97E00E94A807D1E0F0CF0E947B2803
:1043D0006C197D098E099F09693C7105810591055C
:1043E00028F30E947B286B017C01C12719F080ED26
:1043F00097E002C080E090E00E94A807D7CF80E05D
:1044000090E00E94A807DD23B9F08091D30590E0E9
:10441000019665E070E00E94CB2D8093D3050E9449
:104420002B0D0E94A9130E944A0D64EF71E080E0F9
:1044300090E00E94AA2809C080E00E94DF060E9446
:10444000C2110E94410D0E94EF20DF91CF911F9178
:10445000FF90EF90DF90CF90BF90AF909F908F90A4
:104460000895CF92DF92EF92FF9280E00E94DA07E8
:104470000E94B10761E086E00E94342961E085E096
:104480000E94342961E08EE00E94342961E08FE0CF
:104490000E94342960E083E10E94342960E088E0D2
:1044A0000E94342961E088E00E946D290E949F07E4
:1044B00040E052EC61E070E082EE95E00E94CF2C8B
:1044C0000E94A9130E944A0D0E948E138FEF8093C1
:1044D000AA040E94C60778940E947B286B017C0185
:1044E0008091AA048F3F59F40E947B286C197D09A2
:1044F0008E099F09603D77408105910588F380ED25
:1045000097E00E94A80761E083E10E946D295E9A0E
:10451000409A82EE95E00E94872B892B29F082EE4B
:1045200095E00E94B42BF5CF6DEF72E082EE95E03E
:104530000E94422A81E893E00E94300C64E173E01B
:1045400082EE95E00E94422A4AE050E067E070E087
:1045500082EE95E00E94122B62E370E080E090E032
:104560000E94AA2882EE95E00E94872B04970CF106
:1045700082EE95E00E94B42B82349105D1F482EE54
:1045800095E00E94B42B8E34910599F482EE95E06B
:104590000E94B42B8434910561F482EE95E00E9470
:1045A000B42B819731F480E090E00E94A8070E942C
:1045B000EF204091770550917805609179057091D1
:1045C0007A05DB01CA010197A109B1090497A10588
:1045D000B10568F44093A904433029F440EA56E851
:1045E00061E070E004C040E052EC61E070E082EE17
:1045F00095E00E94CF2C0E948B215E98409880E02D
:1046000090E00E94A8070E948E131092C50480912A
:10461000BF0583FF11C080918B05882351F08091E5
:104620009205882331F080919905882311F087E065
:1046300001C085E08093C50480E00E947E0A8091DD
:10464000C6040E94B2090E94590B10923F041092B6
:104650003E0410923D04F12C8091D4058F15B0F0EA
:1046600062E370E080E090E00E94AA2880ED97E08D
:104670000E94A80762E370E080E090E00E94AA2810
:1046800080E090E00E94A807F394E6CF80919E0519
:1046900084FF08C0982F987181E0983109F080E07C
:1046A0000E947E118FE00E94DA07FF90EF90DF906A
:1046B000CF900895EF92FF920F931F93CF93DF93C4
:1046C0008C016EE770E082EE95E00E945906E801E9
:1046D000F12CF0E2EF2E8E0188818D57823048F464
:1046E0006DE770E082EE95E00E94590688818E2584
:1046F00088832196F801608182EE95E00E94E12B8B
:10470000F394F9E0FF12E7CF6EE770E082EE95E0F8
:104710000E945906CDB7DEB7E6E00C94482EA9E01A
:10472000B0E0E5E9F3E20C94302E9091C7049111CA
:104730000EC09EEF99838A836B8350E05595479511
:104740004C832D83198618861F821E822EC04091AD
:10475000CC04842F90E0B4E095958795BA95E1F765
:10476000242F2F7030E08217930719F18DEF898382
:104770001B82FE01349650E0842F90E0A4E09595D2
:104780008795AA95E1F7242F2F7030E082179307C1
:1047900049F0DC01A353BB4F8C918193405F5F5F75
:1047A000563051F74093CC045A83CE0101960E94B3
:1047B0005A238091C70490E0019666E070E00E9461
:1047C000CB2D8093C7042996E2E00C944C2EA0E0F8
:1047D000B0E0EDEEF3E20C94292E6C016EE770E090
:1047E00082EE95E00E9459068601E12CF12CC0E092
:1047F000D0E030E2B32EF801608183E8860F82308A
:1048000078F46DE770E082EE95E00E945906F801B9
:1048100060816B2570E082EE95E00E94590604C02D
:1048200082EE95E00E94E12BE114F10459F0F801C9
:1048300080819E01280F311DC901C92FDD27C80FB6
:10484000D91FDD273FEFE31AF30A89E0E816F104E8
:1048500059F028E0E216F10421F48C2F8095F6013E
:1048600080870F5F1F4FC7CFCDB7DEB7E9E00C944D
:10487000452EA9E0B0E0EFE3F4E20C94302EE82FEF
:10488000362F8091C70490E0019664E270E00E94A8
:10489000CB2D8093C70458E9598350E15A83813066
:1048A00089F048F08230B9F08330D9F48B8381EFFE
:1048B0008C833D8319C085E08B8381EF8C832F5FD0
:1048C0002D8312C08B8381EF8C8384E6489FA001E7
:1048D00011245D8309C084E08B8381EF8C83ED8399
:1048E00003C00E94BB1104C0CE0101960E94E723C1
:1048F0002996E2E00C944C2EA2E0B0E0E2E8F4E26B
:104900000C94252E182F762E2A8349830E948728FF
:104910006B017C018091DD048090C8049090C904F3
:10492000A090CA04B090CB042A8149818823C1F0A9
:10493000D701C60188199909AA09BB094C015D0173
:1049400091EE89169EE29906A104B10420F1241784
:1049500008F4422F202F672D812F0E94392413C085
:10496000D701C60188199909AA09BB094C015D0143
:1049700091E3891695E79906A104B10460F0672DCB
:10498000812F0E948F23C092C804D092C904E09264
:10499000CA04F092CB042296EDE00C94412EA2E2E0
:1049A000B0E0E5EDF4E20C94262E8CE00E9499092B
:1049B00081110FC06CE173E082EE95E00E94732AD2
:1049C0005E9A409A80E00E947E0A0E94590B5E988F
:1049D000409882EE95E00E94872B892B01F182EEB0
:1049E00095E00E94B42B9091A904992319F00E949C
:1049F000BC13EFCF40913E0450E09A012F5F3F4F30
:104A00002F71332760913F0470E02617370709F3B1
:104A1000FA01E75BFB4F808320933E04DACF80915D
:104A20007305843009F086C00E94872861157105DE
:104A30008105910549F06093B7047093B8048093A1
:104A4000B9049093BA040CC081E090E0A0E0B0E01B
:104A50008093B7049093B804A093B904B093BA04B8
:104A60008091AD049091AE0481609093AE048093E8
:104A7000AD0483E0809373058FE70E94770909E610
:104A800014E00E948A09F80181938F01F4E0023753
:104A90001F07B9F72091720480916904982F92271B
:104AA00096FF3BC090E4922790937204982F9873DE
:104AB0009833F1F410E0212F30E080916904877081
:104AC00090E0821793074CF11F5F20919E05812F84
:104AD00090E0FC01E759FB4F24FF04C080810E9455
:104AE0009D11E9CF608182EE95E00E94E12BE3CF3A
:104AF0008F7399F480916A048093B60480916B045B
:104B00008093B40480916C048093B30480916F040B
:104B100090E09093AC048093AB0480913D0481308D
:104B200019F482E080933D0480913D04833011F4B8
:104B300010923D040E9487286B017C018091AF0494
:104B40009091B004A091B104B091B2040097A10576
:104B5000B105C9F0A7019601281B390B4A0B5B0B65
:104B6000DA01C901883B9B40A105B10560F00E94B4
:104B7000C8098093B5041092AF041092B00410924B
:104B8000B1041092B2048091BB049091BC04A09136
:104B9000BD04B091BE0446015701881A990AAA0AB9
:104BA000BB0A86E795E00E94F40786169706A806DA
:104BB000B90608F4A9C0C092BB04D092BC04E0922C
:104BC000BD04F092BE040E9457068091AA0488306A
:104BD000A0F08091BF059091C005A091C105B09152
:104BE000C2056CE1B695A795979587956A95D1F71B
:104BF000892B8A2B8B2B09F0A8C18091AA048F5F87
:104C00008093AA048091B7049091B804A091B9044C
:104C1000B091BA040097A105B105F1F0C81AD90AFC
:104C2000EA0AFB0A86E795E00E94F4076C157D0509
:104C30008E059F0508F008C18091BF0584FD04C062
:104C400080ED97E00E94A8071092B7041092B80474
:104C50001092B9041092BA0490917204907C9093CF
:104C6000720450913E0480913F0420913D045817F6
:104C700009F407C1223009F004C1905890937204DE
:104C8000E0919E05E770F0E0E658FC4F60816930E6
:104C900008F0DFC0615040E04613DDC080933F0460
:104CA00087E3840F90917204892B80937204409360
:104CB000400483E080933D045D9A419A809183058E
:104CC0009091C504911132C10E94790A8091C60465
:104CD0000E94B209E0919E05E770F0E0E658FC4FB3
:104CE000608182E794E00E94940BE091C604EF5F3C
:104CF000E093C604E83109F425C1F0E0EA58FA4F20
:104D00008785882309F41EC10E94030C813069F550
:104D100080919E05887149F18091AD049091AE0417
:104D2000880F991F9093AE048093AD0483E0809325
:104D300073050E94590B0E9487286093AF047093FB
:104D4000B0048093B1049093B204672B682B692B55
:104D500061F481E090E0A0E0B0E08093AF04909334
:104D6000B004A093B104B093B20480919E0584FF77
:104D70001FC08091AD049091AE048E7F0E942A09DD
:104D8000182F6091AB048091B6040E94B213482F93
:104D9000612F8091B50449A30E94B2130091D405FC
:104DA000282F49A16091B3048091B4040E947C240F
:104DB0005D9841988091C3048130C1F018F0823031
:104DC000B1F1D1C083E10E94A029892B09F0CBC0A9
:104DD00081E08093C3040E947B286093BF0470939A
:104DE000C0048093C1049093C204BDC083E10E94BB
:104DF000A029892B31F50E947B28C090BF04D09058
:104E0000C004E090C104F090C2046C197D098E09C1
:104E10009F09693E73408105910508F4A4C082E0B2
:104E20008093C30480ED97E00E94A8079CC083E1B3
:104E30000E94A029892B09F496C080E090E00E948E
:104E4000A8071092C3048FC080E090E00E94A807DA
:104E500003CF68E020CF851709F420CF4F5F242FC0
:104E600030E090E0F901EE58FB4FDC01A75BBB4F4F
:104E70007C917083F901E05CFB4F708301968F7128
:104E80000BCF2430B1F42091400481E494E0A3E7F7
:104E9000B4E0FC013E2F381B321718F431913D93DA
:104EA000F9CF87E3820F90917204892B809372046B
:104EB00000CF8091C304823071F4916090937204AA
:104EC0005E9A409A53ECE52E55E0F52E8E010F5F69
:104ED0001F4FB80111C05E98409880913D04811128
:104EE00003C081E080933D0480913D04833051F7FD
:104EF00084E080933D04E6CFF70181917F0169A3AF
:104F00007AA30E94B415F801819391938F0169A14E
:104F10007AA1F3EDEF16F5E0FF0671F780919E059B
:104F200043E754E087700E947908C6CE882309F4CD
:104F3000CBCE2091C40431E0320F3093C404291346
:104F4000C3CE0DC01092C604DFCE8091AA04883073
:104F500011F45E9A409A89E08093AA04D5CE10920B
:104F6000C4048150B1CEA296ECE00C94422E823063
:104F7000E8F4E82FF0E0EE0FFF1FEB52FA4F7183D9
:104F80006083813041F0809169008C7F842B809315
:104F90006900E89A089580916900440F551F440FF5
:104FA000551F837F842B80936900E99A08951F928F
:104FB0000F920FB60F9211242F933F934F935F934D
:104FC0006F937F938F939F93AF93BF93EF93FF93D1
:104FD0008091D5059091D605892B29F0E091D505D2
:104FE000F091D6050995FF91EF91BF91AF919F91F7
:104FF0008F917F916F915F914F913F912F910F9082
:105000000FBE0F901F9018951F920F920FB60F9220
:1050100011242F933F934F935F936F937F938F93BD
:105020009F93AF93BF93EF93FF938091D705909198
:10503000D805892B29F0E091D705F091D80509957D
:10504000FF91EF91BF91AF919F918F917F916F9160
:105050005F914F913F912F910F900FBE0F901F9036
:1050600018951F920F920FB60F9211242F933F9312
:105070008F939F93AF93BF938091DA059091DB0557
:10508000A091DC05B091DD053091D90523E0230F17
:105090002D3720F40196A11DB11D05C026E8230F70
:1050A0000296A11DB11D2093D9058093DA05909336
:1050B000DB05A093DC05B093DD058091DE059091C2
:1050C000DF05A091E005B091E1050196A11DB11D9C
:1050D0008093DE059093DF05A093E005B093E10592
:1050E000BF91AF919F918F913F912F910F900FBEE4
:1050F0000F901F9018952FB7F8946091DA05709172
:10510000DB058091DC059091DD052FBF08953FB749
:10511000F8948091DE059091DF05A091E005B091B3
:10512000E10526B5A89B05C02F3F19F00196A11DEA
:10513000B11D3FBF6627782F892F9A2F620F711DEF
:10514000811D911D42E0660F771F881F991F4A95A8
:10515000D1F70895CF92DF92EF92FF92CF93DF9332
:105160006B017C010E948728EB01C114D104E1048A
:10517000F10479F00E9487286C1B7D0B683E734018
:10518000A0F381E0C81AD108E108F108C851DC4F4A
:10519000ECCFDF91CF91FF90EF90DF90CF9008950B
:1051A000789484B5826084BD84B5816084BD85B502
:1051B000826085BD85B5816085BDEEE6F0E08081C9
:1051C00081608083E1E8F0E01082808182608083EA
:1051D000808181608083E0E8F0E08081816080836D
:1051E000E1EBF0E0808184608083E0EBF0E080819F
:1051F00081608083EAE7F0E0808184608083808141
:1052000082608083808181608083808180688083E8
:105210001092C1000895833081F028F4813099F014
:105220008230A1F008958630A9F08730B9F084303B
:10523000D1F4809180008F7D03C0809180008F77B2
:1052400080938000089584B58F7702C084B58F7DE8
:1052500084BD08958091B0008F7703C08091B00025
:105260008F7D8093B0000895CF93DF9390E0FC0191
:10527000ED50F44F2491FC01E95FF34F84918823B2
:1052800049F190E0880F991FFC01E15DF34FA59172
:10529000B4918B5D934FFC01C591D4919FB761117F
:1052A00008C0F8948C91209582238C938881822366
:1052B0000AC0623051F4F8948C91322F30958323D8
:1052C0008C938881822B888304C0F8948C91822BE4
:1052D0008C939FBFDF91CF910895A1E0B0E0E3E709
:1052E000F9E20C942E2E282F30E0F901E152F44F10
:1052F0008491F901ED50F44F1491F901E95FF34FF6
:1053000004910023C9F0882321F069830E940B29AE
:105310006981E02FF0E0EE0FFF1FEB5DF34FA591E9
:10532000B4919FB7F8948C91611103C010958123BB
:1053300001C0812B8C939FBF2196E4E00C944A2EF0
:10534000CF93DF93282F30E0F901E152F44F84919D
:10535000F901ED50F44FD491F901E95FF34FC49195
:10536000CC2391F081110E940B29EC2FF0E0EE0F7D
:10537000FF1FE55EF34FA591B4912C912D2381E0A1
:1053800090E021F480E002C080E090E0DF91CF91D6
:1053900008958E3008F08E50877020919D0190E422
:1053A000299F90011124822B80937C0080917A00A8
:1053B000806480937A0080917A0086FDFCCF809192
:1053C00078002091790090E0922B0895A0E0B0E061
:1053D000ECEEF9E20C942A2E6C017A01EB01E60E58
:1053E000F71E00E010E0CE15DF0561F06991D601EF
:1053F000ED91FC910190F081E02DC6010995080F17
:10540000191FF1CFC801CDB7DEB7E8E00C94462EE6
:105410006115710589F0DB010D900020E9F7AD0100
:1054200041505109461B570BDC01ED91FC91028064
:10543000F381E02D0995089580E090E00895EF92C2
:10544000FF920F931F93CF93DF938C01FB01C0E07A
:10545000D0E064917F018FEFE81AF80A662361F0CB
:10546000D801ED91FC910190F081E02DC8010995E2
:10547000C80FD91FF701EDCFCE01CDB7DEB7E6E0FB
:105480000C94482E0E94082A0895DC01ED91FC91AD
:105490000190F081E02D099508950F931F93CF930C
:1054A000DF93EC016DE00E94452A8C016AE0CE0199
:1054B0000E94452A800F911FDF91CF911F910F917C
:1054C00008950F931F93CF93DF93EC010E941F2A3F
:1054D0008C01CE010E944D2A800F911FDF91CF9148
:1054E0001F910F9108950F931F93CF93DF93EC01BA
:1054F0000E94082A8C01CE010E944D2A800F911F24
:10550000DF91CF911F910F9108950F931F93CF9328
:10551000DF93EC010E94452A8C01CE010E944D2AA6
:10552000800F911FDF91CF911F910F910895A1E2FC
:10553000B0E0EDE9FAE20C94262E7C01C42EE52FB2
:10554000CB01D22E19A221E02D1510F02AE0D22E87
:105550008E010F5D1F4F8D2C912CA12CB12C6C2D29
:105560007E2FA50194010E94DF2D8C2DD29E8019E3
:105570001124015011098A3010F4805D01C0895C4A
:10558000F8018083211531054105510521F0C22E16
:10559000E32FCA01E4CFB801C7010E94082AA196EF
:1055A000ECE00C94422EA0E0B0E0E9EDFAE20C94BD
:1055B0002A2EEC016A017B012115310541F4E881B5
:1055C000F9810190F081E02D642F09951DC02A30EA
:1055D0003105A9F477FF12C06DE20E94452A8C01C3
:1055E00044275527BA014C195D096E097F092AE045
:1055F000CE010E94972A800F911F06C02AE0B701B2
:10560000A601CE010E94972ACDB7DEB7E8E00C9440
:10561000462E9A01AB01662757FD6095762F0E94B2
:10562000D32A08950F931F93CF93DF93EC019A0130
:10563000AB01662757FD6095762F0E94D32A8C0117
:10564000CE010E944D2A800F911FDF91CF911F91B3
:105650000F9108952115310549F4DC01ED91FC917C
:105660000190F081E02D642F099508950E94972AFA
:1056700008959A01462F50E060E070E00E942A2BC6
:1056800008959A01AB0160E070E00E942A2B089512
:105690000F931F93CF93DF93EC010E942A2B8C0171
:1056A000CE010E944D2A800F911FDF91CF911F9153
:1056B0000F9108950F931F93CF93DF93EC019A01FD
:1056C000AB0160E070E00E942A2B8C01CE010E94A9
:1056D0004D2A800F911FDF91CF911F910F91089557
:1056E0000F931F93CF93DF93EC019A01462F50E065
:1056F00060E070E00E942A2B8C01CE010E944D2AAE
:10570000800F911FDF91CF911F910F910895FC01A0
:1057100024853585F901E05CFF4F80819181F90195
:10572000EE5BFF4F20813181821B930B8F73992792
:105730000895FC0184859585FC01E05CFF4F408164
:105740005181FC01EE5BFF4F2081318142175307ED
:1057500041F00190F081E02DE80FF91F808190E089
:1057600008958FEF9FEF0895FC0184859585FC01D6
:10577000E05CFF4F40815181FC01EE5BFF4F2081D7
:1057800031814217530779F0A081B181A80FB91F69
:105790008C91208131812F5F3F4F2F7333273183CD
:1057A000208390E008958FEF9FEF0895FC0181A181
:1057B000882329F0A489B5898C9186FFFBCF11A29B
:1057C0000895CF93DF93FC0126853785D901A05C2E
:1057D000BF4F8D919C91119701968F739927E90185
:1057E000CE5BDF4F4881598184179507D9F30D901F
:1057F000BC91A02DA20FB31F6C93A685B785A05CAA
:10580000BF4F11969C938E93A689B7892C9181E006
:1058100090E0078C02C0880F991F0A94E2F7282BAA
:105820002C9381E081A30488F589E02D8081806438
:10583000808381E090E0DF91CF91089508951F92D9
:105840000F920FB60F9211242F933F934F938F9384
:105850009F93EF93FF938091C00082FD1CC0409105
:10586000C600809188069091890601968F739927CA
:1058700020918A0630918B068217930771F0E09190
:105880008806F0918906E85BF94F4083909389067A
:105890008093880602C08091C600FF91EF919F918E
:1058A0008F914F913F912F910F900FBE0F901F90AE
:1058B000189582EE95E00E94872B892B11F00E94AB
:1058C0001E2C08951F920F920FB60F9211242F9342
:1058D0003F938F939F93EF93FF93209144063091D2
:1058E000450680914606909147062817390731F4FE
:1058F0008091C1008F7D8093C10014C0E091460665
:10590000F0914706EC5FF94F208180914606909117
:10591000470601968F739927909347068093460612
:105920002093C600FF91EF919F918F913F912F910E
:105930000F900FBE0F901F901895A0E0B0E0E3EA23
:10594000FCE20C94262EFC011382128288EE93E076
:10595000A0E0B0E084839583A683B7838CEB93E0CB
:10596000918380837587648757874687318B208B27
:10597000138B028BF58AE48AD78AC68AB18EA08EF1
:10598000938E828E8F85848F8889858F8989868F73
:105990008A89878F8B8980A3ECE00C94422ECF926A
:1059A000DF92EF92FF92CF93DF93EC016A017B01CC
:1059B000411581EE580761057105F9F0EC89FD8903
:1059C00081E090E008A002C0880F991F0A94E2F7D6
:1059D000808360E079E08DE390E0A70196010E946A
:1059E000DF2D2150310941095109569547953795C9
:1059F0002795211580E1380798F0EC89FD89108200
:105A000060E874E88EE190E0A70196010E94DF2D26
:105A100021503109410951095695479537952795E8
:105A2000E889F9893083EA89FB89208319A2EE8904
:105A3000FF89408181E090E09C010C8C02C0220F24
:105A4000331F0A94E2F7422B4083EE89FF8940819D
:105A50009C010D8C02C0220F331F0A94E2F7422BE7
:105A60004083EE89FF8940819C010E8C02C0220F89
:105A7000331F0A94E2F7422B4083EE89FF8920818D
:105A80000F8C02C0880F991F0A94E2F78095822339
:105A90008083DF91CF91FF90EF90DF90CF900895BA
:105AA0008F929F92AF92BF92CF92DF92EF92FF922E
:105AB0000F931F9381E08F9385E08F9387E08F93FF
:105AC00083E08F9384E08F93E6EC8E2E912CF2ECA2
:105AD000AF2EB12CA1ECCA2ED12CB0ECEB2EF12CB8
:105AE00004EC10E025EC30E044E056E068E476E0B9
:105AF00082EE95E00E949D2C0F900F900F900F90DA
:105B00000F901F910F91FF90EF90DF90CF90BF907B
:105B1000AF909F908F9008950E94D0280E943122CC
:105B2000C9E5DCE20E94CF242097E1F30E94592CC2
:105B3000F9CFA29FB001B39FC001A39F700D811D3B
:105B40001124911DB29F700D811D1124911D089586
:105B50000E94992DA59F900DB49F900DA49F800D3C
:105B6000911D11240895B7FF0C94A82D0E94A82D13
:105B7000821B930B0895DB018F939F930E94A82DA6
:105B8000BF91AF91A29F800D911DA39F900DB29FD9
:105B9000900D1124089597FB072E16F4009407D05A
:105BA00077FD09D00E945D2E07FC05D03EF490954C
:105BB00081959F4F0895709561957F4F0895A1E25B
:105BC0001A2EAA1BBB1BFD010DC0AA1FBB1FEE1F77
:105BD000FF1FA217B307E407F50720F0A21BB30BC2
:105BE000E40BF50B661F771F881F991F1A9469F73E
:105BF00060957095809590959B01AC01BD01CF019A
:105C00000895052E97FB1EF400940E94182E57FD50
:105C100007D00E94DF2D07FC03D04EF40C94182E01
:105C200050954095309521953F4F4F4F5F4F0895C8
:105C300090958095709561957F4F8F4F9F4F0895F8
:105C40002F923F924F925F926F927F928F929F928C
:105C5000AF92BF92CF92DF92EF92FF920F931F937A
:105C6000CF93DF93CDB7DEB7CA1BDB0B0FB6F8942B
:105C7000DEBF0FBECDBF09942A88398848885F846B
:105C80006E847D848C849B84AA84B984C884DF80DC
:105C9000EE80FD800C811B81AA81B981CE0FD11DC0
:105CA0000FB6F894DEBF0FBECDBFED010895EE0F25
:105CB000FF1F0590F491E02D0994AA1BBB1B51E135
:105CC00007C0AA1FBB1FA617B70710F0A61BB70B6C
:105CD000881F991F5A95A9F780959095BC01CD0111
:105CE00008958F929F92AF92BF92CF92DF92EF92E0
:105CF000FF92CF93DF93EC01688179818A819B8148
:105D0000611571058105910521F464E279ED8BE55A
:105D100097E02DE133EF41E050E00E94012E490170
:105D20005A019B01AC01A7EAB1E40E94A82D6B01C6
:105D30007C01ACEEB4EFA50194010E94B62DC60E15
:105D4000D71EE81EF91EF7FE06C081E0C81AD1086A
:105D5000E10880E8F80AC882D982EA82FB82C7019A
:105D6000B6019F77DF91CF91FF90EF90DF90CF90BA
:105D7000BF90AF909F908F9008950E94712E0895CC
:105D800086E091E00E94712E089560930601709361
:105D90000701809308019093090108952F923F9283
:105DA0005F926F927F928F929F92AF92BF92CF92AB
:105DB000DF92EF92FF920F931F93CF93DF938B01AC
:105DC000EA016115710521F0DB018C9311969C931A
:105DD000209739F09E01225031092332310508F015
:105DE000D8C07C016701BFEFCB1ADB0A5601F7016F
:105DF0006080862D90E00E940030892B11F07601A2
:105E0000F1CFFDE26F120AC0570182E0A80EB11C6B
:105E1000D70111966C90772473940BC0BBE26B1280
:105E200007C05701E2E0AE0EB11CD70111966C908D
:105E3000712CCE018F7E892B89F4B0E36B1237C0B1
:105E4000F50180818F7D8835D1F46180F2E0AF0E5D
:105E5000B11C872D8260782EC0E1D0E0CA30D10518
:105E600051F1C031D10521F0C830D10599F409C0F4
:105E7000CC24CA94DC2CEC2CAFE0FA2E22C0209764
:105E800069F7C8E0D0E0CC24CA94DC2CEC2CFFE10C
:105E9000FF2E17C06FEF7FEFCB019E01442737FD28
:105EA0004095542F0E94DF2D69017A010AC0209786
:105EB000A9F6CAE0D0E0E9E9CE2EDC2CEC2CE9E131
:105EC000FE2EF50160E020E030E0A9014E01AA2499
:105ED00097FCA094BA2C1F0170ED572E560CA9E028
:105EE000A51570F48FEB860D8A3118F499EC592EB4
:105EF00006C08FE9860D8A3148F589EA582E560C7E
:105F0000852D90E08C179D070CF56F3FD9F0C216D8
:105F1000D306E406F50698F0C501B4010E94BB2D36
:105F20009B01AC01852D90E0A0E0B0E0280F391F67
:105F30004A1F5B1F281739074A075B0710F46FEFEA
:105F400001C061E03196D1016C90C5CF01151105FA
:105F500051F0662311F0319703C071FE04C03297EF
:105F6000D801ED93FC9370FE07C050954095309595
:105F700021953F4F4F4F5F4F67FF10C082E290E087
:105F800090938D0680938C066FEF7FEF8FEF9FEFDE
:105F900007C060E070E080E090E002C0B901CA0193
:105FA000DF91CF911F910F91FF90EF90DF90CF90F5
:105FB000BF90AF909F908F907F906F905F903F9039
:105FC0002F900895FC0188279927E8942191203289
:105FD000E9F3293010F02E30C8F32B3241F02D3286
:105FE00039F4689404C00E943430820F911D2191CD
:105FF00020532A30C0F31EF4909581959F4F089549
:10600000911150C0803219F089508550D0F7089511
:1060100048EC53E00E940D300895FA01A191B0813F
:10602000009719F41097E1F0CD01DC01CD010D903E
:10603000002011F4C00113C0FB012191222319F0AB
:106040002015D9F7F3CFFB012191201519F41E92E9
:10605000119606C02223C1F70D900020A1F7D001B0
:10606000FA01A193B08308957AE0979F902D879FBE
:10607000802D910D11240895F999FECF92BD81BD17
:10608000F89A992780B50895262FF999FECF1FBA5F
:1060900092BD81BD20BD0FB6F894FA9AF99A0FBE51
:0E60A00001960895992788270895F894FFCF58
:1060AE0000008E06200001000000FF00020002002A
:1060BE0002000200020002000200020002000200C2
:1060CE00020002000200020002000280250000050C
:1060DE00400AA1204EA50020244EA52C2330C0122C
:1060EE0000001A400AA1204EA5001B1E27522C2389
:1060FE00308025000005400AA1204EA50020244E28
:10610E00A52C2330004B000006400AD0009D49000C
:10611E007B289D492C233000E1000005400A4501F3
:10612E00D7DC03B81E0EBF00232E48E801008A40BC
:10613E000A6001555502AD1E20000023C8015458B7
:10614E002074696D656F75742100596573004E6F0B
:10615E00002C00386368004E2F41002C205B005D40
:10616E002028002900486F70206368616E6E656C90
:10617E00200020402000456E746572696E672061B4
:10618E0064617074697665206368616E6E656C20FB
:10619E0073656C656374696F6E2C207069636B69CF
:1061AE006E673A007363616E6E6572206D6F646523
:1061BE00004E4F5420454E41424C45440053656EAF
:1061CE0064696E672073657474696E677320746F8B
:1061DE002052580A00526573657474696E67207395
:1061EE00657474696E6773206F6E2052580A004191
:1061FE00626F727465642065646974730A00696EF7
:10620E0076616C69642073656C656374696F6E008A
:10621E000D0A496E76616C696420696E7075742022
:10622E002D20646973636172646564210700536590
:10623E007474696E677320736176656420746F2061
:10624E00454550524F4D0A0052657665727465642D
:10625E002073657474696E67732066726F6D204566
:10626E004550524F4D0A004C6F6164656420666163
:10627E0063746F72792064656661756C74730A005D
:10628E004B657920616E64206368616E6E656C7318
:10629E002072616E646F6D697A65640A004F706575
:1062AE006E4C52536E672054582073746172746929
:1062BE006E672000206F6E20485720006D6F64754A
:1062CE006C65206C6F636B65643F00342B34003853
:1062DE0000382B340031320031322B34003136008D
:1062EE0050504D0052535349005344410053434CB8
:1062FE0000525844005458440041494E004C424507
:10630E0045500053504B54524D0053425553005379
:10631E00554D44004C4C494E440000070B0C1011D7
:10632E001500B7012B032F033103350338033D034B
:10633E00B7014003440349034D0351035503590369
:10634E005D0363036A036F0374038D028D028D0276
:10635E008D02160A1322312900000000E12BE629D6
:08636E00872BB42B992BD62BD1
:00000001FF
